:100000000C9401080C9439080C9439080C943908A4
:100010000C9439080C9439080C9439080C9439085C
:100020000C9439080C9439080C942D270C946926EB
:100030000C94F01E0C9439080C9439080C9439086F
:100040000C9439080C9439080C9439080C9439082C
:100050000C9439080C94AF1E0C9439080C94390890
:100060000C9439080C9439080C9439080C9439080C
:100070000C9439080C9439080C9439080C943908FC
:100080000C9439080C9439080C9439080C943908EC
:100090000C9439080C9439080C9439080C943908DC
:1000A0000C9439080C9439080C943908870D870D85
:1000B000B90DB90D2B0E470EDE0FDE0F520E300FAD
:1000C000410F410F8024A7244B26A7244B26F3245D
:1000D00016254B260C261B266261636B6C696768CC
:1000E000742064656372656173653A2025750A0042
:1000F0006261636B6C6967687420696E63726561C5
:1001000073653A2025750A006261636B6C696768E4
:10011000742064697361626C650A006261636B6C70
:100120006967687420656E61626C650A006261636C
:100130006B6C6967687420746F67676C653A20251B
:10014000750A006261636B6C69676874207374651B
:10015000703A2025750A007267626C6967687420BE
:1001600064697361626C65205B454550524F4D5D1B
:100170003A207267626C696768745F636F6E666964
:10018000672E656E61626C65203D2025750A0072E0
:1001900067626C6967687420656E61626C65205B7C
:1001A000454550524F4D5D3A207267626C696768F1
:1001B000745F636F6E6669672E656E61626C652041
:1001C0003D2025750A007267626C69676874207447
:1001D0006F67676C65205B454550524F4D5D3A2017
:1001E0007267626C696768745F636F6E6669672EB9
:1001F000656E61626C65203D2025750A00444542AC
:1002000055473A2064697361626C65642E0A004444
:10021000454255473A20656E61626C65642E0A005E
:1002200053005400550056005F006000610000005C
:100230005C005D005E00570059005A005B005800EA
:1002400062000000630000004F6E6573686F743ACF
:10025000206163746976653A2025640A000A0025E6
:1002600030325820006B6579626F6172645F72652D
:10027000706F72743A20007267626C696768745FAD
:10028000636F6E6669672E7370656564203D202517
:10029000640A007267626C696768745F636F6E6698
:1002A00069672E76616C203D2025640A00726762C2
:1002B0006C696768745F636F6E6669672E736174DB
:1002C000203D2025640A007267626C696768745F6C
:1002D000636F6E6669672E687565203D2025640A28
:1002E000007267686C696768745F636F6E666967E0
:1002F0002E6D6F6465203D2025640A007267626C74
:10030000696768745F636F6E6669672E656E6162A8
:100310006C65203D2025640A007267626C6967681D
:10032000745F636F6E66696720454550524F4D3A62
:100330000A007267626C696768745F696E6974202D
:100340007267626C696768745F636F6E6669672E57
:100350006D6F6465203D20302E20577269746520D2
:1003600064656661756C742076616C756573207464
:100370006F20454550524F4D2E0A007267626C69DE
:100380006768745F696E6974206565636F6E66691E
:1003900067206973206E6F7420656E61626C65649E
:1003A0002E0A007267626C696768745F696E6974AF
:1003B000207374617274210A007267626C696768E5
:1003C000745F696E69742063616C6C65642E0A00E9
:1003D0007267626C696768742064697361626C65D6
:1003E000205B4E4F454550524F4D5D3A207267623B
:1003F0006C696768745F636F6E6669672E656E61AE
:10040000626C65203D2025750A007267626C696721
:10041000687420656E61626C65205B4E4F45455087
:10042000524F4D5D3A207267626C696768745F6312
:100430006F6E6669672E656E61626C65203D202572
:10044000750A005B735D000A0025303862003A20AF
:100450000025303258000A722F6320303132333495
:100460003536370A0000047F3F1F643214643214AB
:10047000783C1E1E140A050A0025303258006C65AF
:10048000645F7461736B3A20006261636B6C6967CF
:1004900068745F636F6E6669672E7261773A2025B4
:1004A0003032580A2E656E61626C653A2025750AF5
:1004B0002E6C6576656C3A2025750A006B65796D42
:1004C00061705F636F6E6669672E7261773A20258F
:1004D0003032580A2E737761705F636F6E74726F7B
:1004E0006C5F636170736C6F636B3A2025750A2EC5
:1004F000636170736C6F636B5F746F5F636F6E7457
:10050000726F6C3A2025750A2E737761705F6C6389
:10051000746C5F6C6775693A2025750A2E73776174
:10052000705F7263746C5F726775693A2025750A33
:100530002E737761705F6C616C745F6C6775693A7C
:100540002025750A2E737761705F72616C745F721B
:100550006775693A2025750A2E6E6F5F6775693A6F
:100560002025750A2E737761705F67726176655F0B
:100570006573633A2025750A2E737761705F626137
:10058000636B736C6173685F6261636B73706163EB
:10059000653A2025750A2E6E6B726F3A2025750A12
:1005A0000064656275675F636F6E6669672E72616E
:1005B000773A20253032580A2E656E61626C653AB2
:1005C0002025750A2E6D61747269783A2025750AA6
:1005D0002E6B6579626F6172643A2025750A2E6D03
:1005E0006F7573653A2025750A006565636F6E66E1
:1005F00069673A0A64656661756C745F6C617965F8
:10060000723A2025750A000A092D204D6167696339
:10061000202D0A443A094465627567204D6573735D
:1006200061676520546F67676C650A583A094D61C8
:1006300074726978204465627567204D6F64652027
:10064000546F67676C65202D2053686F77206B654A
:10065000797072657373657320696E206D61747251
:10066000697820677269640A4B3A094B6579626F51
:1006700061726420446562756720546F67676C65BA
:10068000202D2053686F77206B65797072657373C6
:10069000207265706F72740A4D3A0944656275671D
:1006A000204D6F75736520546F67676C650A563A05
:1006B0000956657273696F6E0A533A09537461740F
:1006C00075730A433A09416374697661746520431E
:1006D0006F6E736F6C65204D6F64650A46312D46F1
:1006E00031303A0953776974636820746F204C6124
:1006F00079657220302D392028463130203D204C3C
:1007000030290A302D393A095377697463682074A7
:100710006F204C6179657220302D390A475241565D
:10072000453A0953776974636820746F204C617986
:10073000657220302028616C7465726E6174652961
:100740000A423A094A756D7020746F20426F6F74C7
:100750006C6F616465720A4553433A094A756D705E
:1007600020746F20426F6F746C6F61646572202813
:10077000616C7465726E617465290A453A0950723C
:10078000696E7420454550524F4D2053657474690D
:100790006E67730A4253504143453A09436C6561A1
:1007A0007220454550524F4D0A000A092D20436FD3
:1007B0006E736F6C65202D0A4553432F713A097192
:1007C0007569740A6D3A096D6F7573656B65790AA1
:1007D000000A092D2056657273696F6E202D0A5626
:1007E00049443A2030783530353328506572636596
:1007F0006E742053747564696F29205049443A20FF
:1008000030783432353328426F6F73746572292023
:100810005645523A203078303030310A4255494CF2
:10082000443A202028466562203238203230323265
:10083000290A4F5054494F4E533A204C55464120B7
:100840004D4F5553454B45592045585452414B4502
:100850005920434F4E534F4C4520434F4D4D414E31
:1008600044204C544F20343039360A4743433A2011
:10087000352E342E30204156522D4C4942433A20D9
:10088000322E302E30204156525F415243483A209A
:10089000617672350A000A092D20537461747573EC
:1008A000202D0A686F73745F6B6579626F61726483
:1008B0005F6C65647328293A20253032580A6B65CD
:1008C00079626F6172645F70726F746F636F6C3A9C
:1008D00020253032580A6B6579626F6172645F69F6
:1008E000646C653A20253032580A74696D65725F10
:1008F00072656164333228293A202530386C580AF1
:10090000003F000A6D6F7573653A206F66660A00D6
:100910000A6D6F7573653A206F6E0A000A6B657910
:10092000626F6172643A206F66660A000A6B6579CD
:10093000626F6172643A206F6E0A000A6D617472B0
:1009400069783A206F66660A000A6D617472697888
:100950003A206F6E0A000A64656275673A206F6616
:10096000660A000A64656275673A206F6E0A000ABB
:100970000A4A756D70696E6720746F20626F6F74BC
:100980006C6F616465722E2E2E2000433E20004362
:100990006C656172696E6720454550524F4D0A0083
:1009A000313A0964656C6179282A31306D73293ACE
:1009B0002025750A323A09696E74657276616C2871
:1009C0006D73293A2025750A333A096D61785F7392
:1009D000706565643A2025750A343A0974696D6555
:1009E0005F746F5F6D61783A2025750A353A097733
:1009F0006865656C5F6D61785F73706565643A20EA
:100A000025750A363A09776865656C5F74696D65A6
:100A10005F746F5F6D61783A2025750A00703A093E
:100A20007072696E742076616C7565730A643A0938
:100A30007365742064656661756C74730A75703AC9
:100A4000092B310A646E3A092D310A6C743A092B6C
:100A500031300A72743A092D31300A4553432F71EF
:100A60003A09717569740A0A7370656564203D20DE
:100A700064656C7461202A206D61785F73706565B0
:100A800064202A2028726570656174202F207469A3
:100A90006D655F746F5F6D6178290A77686572654F
:100AA0002064656C74613A20637572736F723D25C2
:100AB000642C20776865656C3D25640A5365652064
:100AC000687474703A2F2F656E2E77696B69706544
:100AD0006469612E6F72672F77696B692F4D6F752F
:100AE00073655F6B6579730A004D3E20004D257577
:100AF0003A25733E20003F0A003D2025750A003F3D
:100B00000A0064656661756C74730A0025750A00D5
:100B10003F0A000A092D2056616C756573202D0A65
:100B200000710A000A092D204D6F7573656B657998
:100B3000202D0A004C25640A000631FF0974A1012A
:100B40000975150026FF00952075088102097615A4
:100B50000026FF00952075089102C005010902A139
:100B60000185020901A100050919012908150025BF
:100B700001950875018102050109300931158125AA
:100B80007F95027508810609381581257F950175C5
:100B9000088106050C0A38021581257F9501750824
:100BA0008106C0C005010980A101850319012AB78A
:100BB00000150126B700950175108100C0050C09CC
:100BC00001A101850419012AA002150126A00295A0
:100BD0000175108100C005010906A101050719E092
:100BE00029E7150025019508750181029501750811
:100BF00081010507190029FF150026FF00950675DC
:100C000008810005081901290595057501910295CE
:100C10000175039101C05B435D005B445D005B5364
:100C20005D005B575D005B525D0009025B000301E4
:100C300000A0FA09040000010301010009211101CB
:100C4000000122400007058103080001090401009A
:100C50000103000000092111010001227B000705AA
:100C600082032000010904020002030000000921A0
:100C7000110100012222000705830320000107055E
:100C8000030320000112010002000000085350532A
:100C900042010001020001100342006F006F007367
:100CA0000074006500720000001E035000650072B1
:100CB00000630065006E007400200053007400752E
:100CC00000640069006F0000000403090472676299
:100CD0006C696768742073657420687376205B4E56
:100CE0004F454550524F4D5D3A2025752C25752CAA
:100CF00025750A007267626C696768742073657491
:100D000020687376205B454550524F4D5D3A202553
:100D1000752C25752C25750A007267626C696768E9
:100D200074207261696E626F7720736574206873D6
:100D3000763A2025642C25642C25642C25750A0020
:100D4000FFAA7F55407267626C6967687420746996
:100D50006D657220656E61626C65642E0A00726753
:100D6000626C696768742074696D65722064697368
:100D700061626C652E0A002223252628292A2C2D43
:100D80002F3032333536383A3B3D3E4042434547BB
:100D9000494A4C4E5051535557595A5C5E606264F3
:100DA0006668696B6D6F71737577797B7D7F818301
:100DB0008587898A8C8E90929496989A9C9E9FA102
:100DC000A3A5A7A8AAACAEAFB1B3B4B6B8B9BBBC23
:100DD000BEBFC1C2C3C5C6C7C9CACBCCCDCED0D198
:100DE000D2D2D3D4D5D6D7D7D8D9D9DADADBDBDB90
:100DF000DCDCDCDCDCDDDDDDDDDCDCDCDCDCDBDB31
:100E0000DBDADAD9D9D8D7D7D6D5D4D3D2D2D1D084
:100E1000CECDCCCBCAC9C7C6C5C3C2C1BFBEBCBB81
:100E2000B9B8B6B4B3B1AFAEACAAA8A7A5A3A19FF9
:100E30009E9C9A98969492908E8C8A8987858381BD
:100E40007F7D7B79777573716F6D6B69686664629E
:100E5000605E5C5A5957555351504E4C4A4947456C
:100E60004342403E3D3B3A3836353332302F2D2C0D
:100E70002A292826252322290A002575002F002546
:100E800075005D28002564002000256400200025F1
:100E9000640020002564007C0025303258006D6F0E
:100EA0007573656B6579205B62746E7C7820792040
:100EB0007620685D287265702F61636C293A205B2B
:100EC000000001010101010101010102020202020F
:100ED00002020202030303030303030304040404E2
:100EE00004040405050505050606060606070707AA
:100EF000070708080808090909090A0A0A0B0B0B61
:100F00000C0C0C0D0D0D0E0E0E0F0F0F10101111FD
:100F10001112121313141415151616171718181981
:100F2000191A1A1B1B1C1D1D1E1E1F2020212222E8
:100F3000232424252626272829292A2B2C2D2D2E2B
:100F40002F30313232333435363738393A3B3C3D45
:100F50003E3F404142434445464748494A4C4D4E36
:100F60004F50515354555658595A5B5D5E5F6162FC
:100F700064656668696B6C6D6F7072737577787A8B
:100F80007B7D7E8082838587888A8C8E8F919395E6
:100F900096989A9C9EA0A2A3A5A7A9ABADAFB1B30A
:100FA000B5B7BABCBEC0C2C4C6C9CBCDCFD1D4D6EA
:100FB000D8DBDDDFE2E4E7E9EBEEF0F3F5F8FAFD8C
:100FC000FF7267626C69676874206D6F6465205B8F
:100FD0004E4F454550524F4D5D3A2025750A0072DF
:100FE00067626C69676874206D6F6465205B454556
:100FF00050524F4D5D3A2025750A003F00433E2078
:10100000000011241FBECFEFDAE0DEBFCDBF04B673
:1010100003FE18C08091D8029091D902A091DA0203
:10102000B091DB028730904BA740B04B59F410923F
:10103000D8021092D9021092DA021092DB02E0E09C
:10104000F8E3099511E0A0E0B1E0E6E0F6E602C0C1
:1010500005900D92AC3EB107D9F722E0ACEEB1E0BD
:1010600001C01D92A83DB207E1F70E94A9170C9498
:1010700001330C940000FF93EF93E091EC01F091A9
:10108000ED01309709F00995EF91FF910895FC016A
:101090008591803011F0EFDFFBCF0895FF27E0E26C
:1010A00030E247FF0CC0419597FF09C0EDE2609523
:1010B000709580959095611D711D811D911D27FF73
:1010C00002C0219530E350E2AA27660F771F881FE0
:1010D000991FAA1FA41710F0A41B63955A95A9F78E
:1010E000AA3008F0A95FA05DAF93F3956115710573
:1010F0008105910541F7ED3211F4EF93F395F21765
:1011000018F43F93F395FBCF8F91B5DFFA95E1F794
:101110000895E991F9918591803021F0853219F097
:10112000AADFF9CF089520E0E89455915532C1F334
:10113000503311F4689455915A3348F4505390F356
:10114000220F022E220F220F200D250FF4CF0EF4B6
:10115000219589919991533619F3533729F15335D4
:1011600059F1BC0188279927E8945C3621F48991CC
:10117000999168945591543639F446EF7EF077FF93
:101180000DC08FEF9FEF0AC055374AE039F0583550
:1011900040E121F0523642E009F00895FF93EF93C9
:1011A0007DDFEF91FF91B7CFFF93EF93FC0181912A
:1011B0008030B9F360DFFBCFFF93EF9368DFF1CFAF
:1011C000DF93CF93CDB7DEB72596A3DFCF91DF9125
:1011D00008951F93CF93DF93CDB7DEB767970FB610
:1011E000F894DEBF0FBECDBF4B8B5C8B6D8B7E8BBF
:1011F0008F8B61111092380286E09E01235F3F4F72
:10120000D901E82F1D92EA95E9F795E0FE01739662
:10121000D90101900D929A95E1F79C894E895F89D9
:101220007B897D879E876F87598B488BF901DE010B
:10123000179601900D928A95E1F7CE0107960E94CC
:10124000081681113EC086E0FE013796DE01119638
:1012500001900D928A95E1F7FF81E8856A857B858B
:101260006115710531F0EF3F31F481E0FF3F19F472
:1012700003C081E001C080E080FD23C02091FD011A
:1012800030E0C90101968770992740912E0250E005
:101290008417950779F1F983EA837D836C8396E05F
:1012A000929FD001939FB00D1124A250BE4FFE011A
:1012B000319601900D929A95E1F78093FD010E947D
:1012C000741516E080912E029091FD018917F9F0B6
:1012D000189FC001112482509E4F0E940816882337
:1012E000B1F080912E0290E001968770992780934B
:1012F0002E02E8CF0E94FC301092FD0110922E02C7
:10130000E7EFF1E086E0DF011D928A95E9F7679645
:101310000FB6F894DEBF0FBECDBFDF91CF911F9106
:1013200008958F929F92AF92BF92CF92DF92EF92E9
:10133000FF920F931F93CF93DF93CDB7DEB72A971A
:101340000FB6F894DEBF0FBECDBFFC01D080118177
:1013500083819481892B39F01F3F39F491E00FEF9D
:10136000D01203C003C091E001C090E090FD8CC793
:101370007F0185E0DE01169601900D928A95E1F7D6
:10138000F70122818E819F81222349F00E94D22F72
:10139000082F682F8E819F810E94583003C00E94C1
:1013A0002D30082FE12FF0E015E0019FE00DF11D39
:1013B0001124EE0FFF1FEE0FFF1FED0DF11DEE0FBD
:1013C000FF1FE05EFD4F05911491F7018281882394
:1013D00009F414C10E3BFCE51F07B9F188F40C3B7E
:1013E0003CE51307D1F00D3B9CE5190709F006C158
:1013F0008091BB0287708E7F8093BB0280E01EC00D
:10140000003CECE51E0709F473C008F447C0013C3A
:101410002CE5120709F4B5C0F1C08091BB028770BA
:1014200088618093BB02887F91E009F490E080910D
:10143000BB0290FB80F98093BB0283E00E94B7223D
:101440008091BB020E946A230EC68091BB02982F36
:10145000969596959695A1F0915E990F990F990F93
:101460008770892B8093BB02887F91E009F490E01C
:101470008091BB0290FB80F98093BB020E946A239B
:1014800080915C0280FFB4C08091BB0286958695F6
:1014900086951F928F9388ED90E0A2C02091BB02A9
:1014A000822F869586958695482F50E043305105CA
:1014B00054F48F5F982F990F990F990F822F87708F
:1014C000892B8093BB028091BB0281608093BB0219
:1014D0000E946A2380915C0280FF8AC08091BB02D7
:1014E0008695869586951F928F9380EF90E078C0C1
:1014F0001091BB02117080915C0280FF0CC01F92A2
:101500001F938DE291E09F938F930E94E0080F90CC
:101510000F900F900F908091BB021123B9F080FFC4
:10152000A2C58E7F8093BB020E946A2380915C02D9
:1015300080FF08C088E091E09F938F930E94E008AD
:101540000F900F9080E00E94B7228DC580FD8BC563
:1015500081608093BB02813019F489E08093BB02E3
:101560008091BB020E946A2380915C0280FF40C090
:101570008BE191E09F938F930E94E0080F900F9072
:1015800037C09091BB02892F8695869586958F5F8F
:101590008F719770843038F4880F880F880F892BEB
:1015A0008093BB0202C09093BB028091BB02887FF4
:1015B00091E009F490E08091BB0290FB80F9809368
:1015C000BB020E946A2380915C0280FF11C080915F
:1015D000BB028695869586951F928F9383E491E052
:1015E0009F938F930E94E0080F900F900F900F90A1
:1015F0008091BB02869586958695A5CF043F2CE504
:10160000120799F406E221EE40EE64EF7CE509C092
:10161000083DFCE51F0711F506E221EE41EE68EDFD
:101620007CE5C7010E946B1F1EC5053F3CE5130703
:1016300008F05CC1093D9CE5190731F407E225EE8D
:1016400045EE69ED7CE5EDCF0A3DECE51E0701F7BF
:1016500008E221E045EE6AED7CE5E3CF882309F45A
:101660007AC11092640204303DE5130758F40B3F31
:101670008CE5180780F4C80182509C45449708F017
:1016800054C109C002369DE5190729F0063AEDE577
:101690001E0709F04AC10E94251490934C028093C2
:1016A0004B020131FCE51F0709F4C6C008F042C037
:1016B00009303CE5130709F49BC000F505309CE5B3
:1016C000190709F485C078F40330FCE51F0709F415
:1016D00078C008F07AC002301C4509F0F7C080914C
:1016E0004B028160F1C007308CE5180709F478C01F
:1016F00008F07AC080914B028061E6C00D30ECE5C5
:101700001E0709F487C058F40B302CE5120709F4C2
:1017100079C008F07BC080914B0288606FC00F30A9
:101720008CE5180709F480C008F082C080914B0254
:10173000877FCAC00E3FECE51E0709F471C000F5B3
:1017400005312CE5120709F485C068F403318CE5F6
:10175000180709F475C008F095C00E94FC3080910C
:101760004B028F77B1C00C3FECE51E07A9F108F0E2
:1017700054C00B3F1C4509F0A9C080914C0240C0E9
:1017800002303DE5130709F489C058F401159DE5C1
:10179000190709F45AC008F069C080914C028260B0
:1017A0002FC00236FDE51F0709F47EC0063A2DE57D
:1017B000120709F483C003301D4509F087C060E0BB
:1017C0006EC080914B0282607FC080914B0216C038
:1017D00080914B02886078C080914C0282604FC03B
:1017E00080914B02806270C080914B0280646CC01B
:1017F0000E94FC3080914B02806866C0846064C0A7
:1018000081603DC080914B028E7F5EC080914B0213
:101810008D7F5AC080914B0216C080914C0218C037
:1018200080914C028D7F2BC080914B028F7E4CC0EB
:1018300080914B028F7D48C080914B028F7B44C0CA
:1018400080914B02877F8B7F3FC080914C028D7FC0
:101850008E7F15C080914B0282FB222720F991E0F8
:10186000922790FB82F990FB83F92EC080914C0265
:10187000982F909591708E7F892B90FB81F98093A2
:101880004C0224C00E94FC3080914B0287FB22272F
:1018900020F991E0922790FB87F916C061E08EE075
:1018A00090E00E94083212C080914B0284FB2227F4
:1018B00020F991E0922790FB84F906C080914B02B9
:1018C000982F909590FB80F980934B0260914B028A
:1018D00010914C0284E090E00E940832612F82E275
:1018E00090E00E9408320E94FC30BDC3063F2CE508
:1018F000120731F406E221EE42EE66EF7CE591CE6E
:10190000063F3CE5130730F407E225EE44EE65EFB1
:101910007CE587CE073F9CE5190709F09FCE07E2DB
:1019200025EE46EE67EF7CE57CCE0631ECE51E0742
:1019300061F5809139028A7A91E009F490E0909300
:10194000EE01882311F065E301C069E28FEE91E0BA
:101950000E94191F17C00631FCE51F0709F060C07F
:101960008091EE01882309F4A1C385E3EFEEF1E055
:1019700025EF31E09281891301C0128231962E1732
:101980003F07C1F70E94AE146EC30F3DFCE51F0771
:10199000C1F140F401153CE5130791F001301C45FD
:1019A000E9F05AC00C359DE51907B1F10D35EDE5AB
:1019B0001E0751F10B351D4509F04EC081E02DC0C9
:1019C0000E94FC300FEF14E32CE001501040204047
:1019D000E1F700C000000E948B1E45C380915C02AD
:1019E000982F9095917090FB80F980935C029923D9
:1019F00019F08FE092E002C08DEF91E00E9447085D
:101A000032C30E9436142FC380914C0282FB882778
:101A100080F991E0892701C080E00E9445151CC033
:101A20008091390282720D3C9CE5190709F40CC4BF
:101A300008F002C3073CFCE51F0709F4F1C308F0F6
:101A400045C3043C3CE5130709F4E0C308F030C388
:101A5000033C1C4509F47BC3F7018281008111819D
:101A6000882349F0C8010E94D22FD82E682FC801C0
:101A70000E94583004C0C8010E942D30D82EE12F9A
:101A8000F0E015E0D19EE00DF11D1124EE0FFF1FD7
:101A9000EE0FFF1FE00FF11DEE0FFF1FE05EFD4F89
:101AA000859194910E948B128C01982EF701D2801F
:101AB000A580A2945FE0A52280912F028770B9F0E3
:101AC000DD20A9F0812F807F803421F080E2800F1B
:101AD000883068F080914C0282FD09C082E00E944B
:101AE000281580912F028770CC24C3948111C12CBA
:101AF000B12EB2942FE0B2228B2D90E08C30910564
:101B000008F05CC2FC01EA5AFF4F0C94B032812FFE
:101B1000807F1F70882311F01295107FDD20B9F0AF
:101B2000112309F438C280E2800F883010F0911040
:101B300006C080913902182B1093390205C080919C
:101B40003802182B109338020E94AE1424C2802F42
:101B50000E941831112309F431C2005E083078F177
:101B6000992069F11095809138021823109338025A
:101B700029C0812F807F1F70803211F01295107F55
:101B8000992021F0F1E09F16D9F149C080914C02D3
:101B900082FF1BC0DD2069F0112339F080913902EA
:101BA000182B109339020E94AE1480E00E9450312D
:101BB00005C280E00E941831112309F4FFC1812F72
:101BC0000E94A7140E94AE14F9C1DD2081F080911B
:101BD0003A02AA2051F001E0A01207C0182B1817F2
:101BE00009F4ECC110933A02E9C1812B10C0AA207C
:101BF00021F021E0A21609F4E1C10E94A11427C03E
:101C0000DD2041F035E03A1508F4D8C1812F0E945B
:101C10000E31D4C184E08A1508F4D0C118C0DD208B
:101C200049F0AA2099F3F701858180FFB4C18F7034
:101C30008583ECCFAA2059F0093309F0BCC1FFEF2E
:101C400017EE23E0F15010402040E1F7B2C1812FA0
:101C50000E940731B3C1812F86958695837019F054
:101C6000813059F0ABC1DD2019F0C801937002C07A
:101C700080E090E00E94491FA7C1DD2019F0C80153
:101C8000937002C080E090E00E94331F9DC1802FBE
:101C9000DD2019F00E945C2F02C00E946D2E0E9470
:101CA000C12D92C1812F837009F069C0D1108AC102
:101CB000902F929596959770990F990F802F8F700E
:101CC000882E912CA12CB12C092E04C0880C991CB3
:101CD000AA1CBB1C0A94D2F704FF12C04FE050E0CC
:101CE00060E070E004C0440F551F661F771F9A958F
:101CF000D2F7DB01CA0180959095A095B09503C0FD
:101D000080E090E0DC0116951695412F437042303B
:101D100019F1C8F400913B0210913C0220913D0260
:101D200030913E02413059F088299929AA29BB29CE
:101D3000BC01CD0160237123822393230AC0802A32
:101D4000912AA22AB32ABC01CD01682979298A29BE
:101D50009B290E94D23036C188299929AA29BB29FA
:101D600000913B0210913C0220913D0230913E02D5
:101D7000BC01CD016027712782279327EACFDD20A0
:101D800019F0812F817001C08695882309F41AC14A
:101D9000902F929596959770990F990F802F8F702D
:101DA000882E912CA12CB12C092E04C0880C991CD2
:101DB000AA1CBB1C0A94D2F704FF12C04FE050E0EB
:101DC00060E070E004C0440F551F661F771F9A95AE
:101DD000D2F7DB01CA0180959095A095B09503C01C
:101DE00080E090E0DC0116951695412F437042305B
:101DF000D9F068F5009147021091480220914902FC
:101E000030914A02413059F088299929AA29BB29E1
:101E1000BC01CD0160237123822393231EC0802A3D
:101E2000912AA22AB32A13C088299929AA29BB2951
:101E300000914702109148022091490230914A02D4
:101E4000BC01CD01602771278227932706C0BC0102
:101E5000CD01682979298A299B290E948230B2C044
:101E60001F70DD2039F0812F0E94B130802F0E9439
:101E70000E31A8C0802F0E940731812F0E948C3024
:101E8000A1C0802F32EF931609F443C0391538F002
:101E900090EF991659F0E1EF9E16B1F177C0F3EF8C
:101EA0009F16F1F124EF921659F170C0DD2019F15F
:101EB00034E03A1508F482C01F7181E090E0A0E0A0
:101EC000B0E0AC01BD0104C0440F551F661F771F71
:101ED0001A95D2F78091470290914802A091490249
:101EE000B0914A028A019B01082719272A273B271C
:101EF000C901B80129C025E02A1508F45FC0DCCF6C
:101F000080914C0282FF23C0DD2029F0812F8F7148
:101F100030C0DD20D9F3812F8F710E948C304EC0EC
:101F2000DD2079F01F7181E090E0A0E0B0E0BC011D
:101F3000CD0104C0660F771F881F991F1A95D2F72D
:101F400003C060E070E0CB010E94823037C0DD202A
:101F500099F01F71812F0E94B13080914C0282FD57
:101F600007C038E0139FC0011124836080932F02C3
:101F7000812F0E94B13022C081E00E94281581E0AB
:101F80008A15E0F482E00E94281518C0DD2029F0AF
:101F9000AA2009F4BBCF802F09CEAA2009F4BBCF19
:101FA000893349F49FEFE7EEF3E09150E040F040D1
:101FB000E1F700C00000802F0E94183188EF8B0DE0
:101FC000843010F40E945F1FCC20A9F080912F0272
:101FD00080FD11C0F70112828595859585950E9437
:101FE000B130C7010E94910980912F028595859596
:101FF00085950E948C3085E0F701DE0111960190F5
:102000000D928A95E1F789819A810E942D30EA81AB
:10201000F0E005E0809FE00DF11D1124EE0FFF1FA1
:10202000EE0FFF1F8981E80FF11DEE0FFF1FE05E2D
:10203000FD4F8591949128C1023D8CE5180709F464
:1020400013C108F465C0053D8CE5180709F412C1F9
:1020500008F471C0063D2CE5120709F410C10E35D5
:102060001D4509F0F9CC80912F02877009F40CC14D
:10207000F7018281882309F407C180914C0282FD17
:1020800003C182E02A960FB6F894DEBF0FBECDBF23
:10209000DF91CF911F910F91FF90EF90DF90CF9044
:1020A000BF90AF909F908F900C94281589E25ECCE2
:1020B000053CFCE51F0709F4AEC0063C1C4509F0D1
:1020C000CBCC48E75CE261E87CE2C2C00A3C3CE57C
:1020D000130709F4AFC070F4083CECE51E0709F4DF
:1020E000A4C0093C1C4509F0B7CC4CE65CE260E6B4
:1020F0007CE2AEC00B3C2CE5120709F4A0C00C3CFE
:102100001C4509F0A9CC49E558E26AE678E2A0C08E
:102110000F3CECE51E0709F4A1C008F49CC0003D8B
:102120002CE5120709F49DC0013D1C4509F094CC33
:102130006EE089E0A1C0033DECE51E0709F497C0FD
:10214000043D1C4509F088CC61E088E19AC080918B
:102150005C0280FF10C08091B602809581701F9252
:102160008F9386EC91E09F938F930E94E0080F90ED
:102170000F900F900F908091B60280FF2EC08E7F3F
:102180008093B6026091B6027091B7028091B80256
:102190009091B9020E949D2C80915C0280FF0FC03B
:1021A0008091B60281701F928F9387E591E09F9393
:1021B0008F930E94E0080F900F900F900F900E9455
:1021C000C1288FEF90E7E2E081509040E040E1F7D6
:1021D00000C000000E94F22846CF81608093B602C2
:1021E00080915C0280FF0DC01F9281E08F938FE889
:1021F00091E09F938F930E94E0080F900F900F90B3
:102200000F908091B60261E086953BC049E05DE2A7
:1022100062E17DE21DC042E15DE269E07DE218C05D
:1022200041E85CE268E77CE213C040E65CE26CE611
:102230007CE20EC048E45CE264E57CE209C044E56F
:102240005CE268E47CE204C04AE658E269E578E2D0
:102250000E94BB2808CF61E081E013C065E082E006
:102260000BC068E086E008C064E18FE005C067E16C
:1022700085E102C062E289E10E94A928F4CE61E012
:1022800083E20E94AF2CEFCE2A960FB6F894DEBF01
:102290000FBECDBFDF91CF911F910F91FF90EF90B7
:1022A000DF90CF90BF90AF909F908F9008958295D0
:1022B000982F937344E0949F900111248C7C869511
:1022C0008695282B822F8575880F2A7A2695822B52
:1022D000089590914B0292FF0DC0282F287128304D
:1022E00019F4877F846006C0282F2471243011F4EC
:1022F0008B7F886093FF0DC0282F2871283119F437
:10230000877E846106C0282F2471243111F48B7ECE
:10231000886120914C0220FF0DC0382F3871383071
:1023200019F4877F816006C0382F3171313011F484
:102330008E7F886021FF0DC0282F2871283119F465
:10234000877E816106C0282F2171213111F48E7E94
:10235000886194FD877E0895F894E82FE295EF70E8
:10236000F0E031A1282F2F7081E090E001C0880FAC
:102370002A95EAF7982F9095932391A392A1892B00
:1023800082A3789408957F928F929F92AF92BF928A
:10239000CF92DF92EF92FF920F931F93CF93DF9331
:1023A00000D000D01F92CDB7DEB7AE014F5F5F4FB8
:1023B0007A0185E0FA0111928A95E9F702E511E0C8
:1023C0006A0187E5A82E81E0B82E88248394912C99
:1023D000F80180818F3F09F441C0F894E82FE2951D
:1023E000EF70F0E021A18F70A40102C0440F551FCF
:1023F0008A95E2F7CA01922F982B91A392A180951A
:10240000892382A3789400C0E7E5F1E0712C31E0E4
:1024100021912F3F89F0A22FA295AF70B0E0909646
:102420008C9190E02F7002C0959587952A95E2F7E0
:1024300080FD02C0832F01C080E0782A330F51E075
:10244000EB35F50729F7F80180818F3F11F00E94E5
:10245000AC11F0EAFA95F1F7F60170820F5F1F4FA9
:10246000FFEFCF1ADF0AA016B10609F0B1CF45E0A1
:1024700050E0B70182E492E00E94F43211E000974C
:1024800009F410E0892B89F085E0F701A2E4B2E0BD
:1024900001900D928A95E1F781E0809341020E94BC
:1024A000E41E9093400280933F0280914102882372
:1024B000F1F080913F02909140020E94D51E059755
:1024C000B0F0809142028093500280914302809349
:1024D0005102809144028093520280914502809380
:1024E0005302809146028093540210924102812F40
:1024F0000F900F900F900F900F90DF91CF911F9141
:102500000F91FF90EF90DF90CF90BF90AF909F9092
:102510008F907F900895CF93DF938238910569F172
:10252000B0F48133910509F46FC048F48932910504
:1025300009F465C08A32910509F46BC08AC08533FD
:10254000910509F457C089339105B9F082C0833EE3
:10255000910571F138F4803E9105B1F0823E91050C
:1025600011F177C0863E9105B9F1873E9105C9F119
:10257000843E910509F06DC024C020914B0220FDDE
:1025800053C021FD51C065C080914B0280FD46C003
:1025900080914C0280FF48C080914B0284FD50C165
:1025A00083EE90E04FC180914B0282FF3AC0F4CF9E
:1025B00080914B0282FD35C080914C0280FD34C079
:1025C000EBCF80914C0281FF35C080914B0284FD9E
:1025D00037C187EE90E036C180914B0283FF27C060
:1025E000F4CF80914B0283FD22C080914C0281FD8B
:1025F00021C0EBCF80914B0285FD1FC021C080918F
:102600004B0285FD1DC019C080914B0286FD1BC089
:102610001DC080914B0286FD19C015C089E390E072
:1026200011C182EE90E00EC180EE90E00BC186EE0B
:1026300090E008C184EE90E005C189E290E002C11B
:1026400085E390E0FFC08AE290E0FCC081E390E087
:10265000F9C0811531E5930708F069C0811540E59F
:102660009407F0F09C0174E0369527957A95E1F790
:10267000922F9370482F437021E030E002C0220F68
:10268000331F4A95E2F73C68392B982F9F70969537
:10269000969540E2949FC0011124822B932BD2C0C7
:1026A000883E910568F5803E910508F0CBC0883AD8
:1026B0009105B8F4853A910548F0855AE82FF0E085
:1026C000EF5DFE4F808190E09064BCC08130910549
:1026D00009F4B3C008F4B4C08430910508F4B0C064
:1026E000B1C08F3B910508F0ABC0885AE82FF0E0ED
:1026F000EE0FFF1FEC5DFE4F808191819464A2C0BC
:10270000811520E2920758F4811531E0930708F013
:1027100099C08D3E910508F493C0906593C08115D2
:1027200040E4940708F48CC09F70906A8BC08115B8
:1027300025E5920708F042C0811534E5930728F09B
:10274000982F8827846F906A7DC0811543E5940790
:10275000B0F09C012370332741E050E002C0440FE9
:10276000551F2A95E2F7282F2695269580E2289F67
:1027700090011124CA01822B932B9A6863C08115A2
:1027800022E5920728F4982F8827816F906A5AC013
:102790009C012370332741E050E002C0440F551FD5
:1027A0002A95E2F7282F2695269580E2289F90010A
:1027B0001124CA01822B932B9C6844C0EC01811523
:1027C00039E59307A8F48115984528F09C2F8827B0
:1027D000806F906A37C0C11586E5D80788F58C2FC1
:1027E0000E9469118F7190E0982F882790622AC00B
:1027F00081152AE5920790F48C2F8F700E94691141
:1028000094E0D695C7959A95E1F7CF70D0E0DC2F8C
:10281000CC27D0699E01282BC90114C09056811580
:10282000904270F48D2F8F710E946911282F2F71A3
:10283000CE0199279062922B05C081E090E002C002
:1028400080E090E0DF91CF910895CF9384E090E015
:102850000E94F431C82F82E290E00E94F4312C2FC4
:1028600030E0A901582BCA01CF91089569EE7EEF9F
:1028700080E090E00E94263260E082E090E00E94DA
:10288000083260E083E090E00E94083210923B0240
:1028900010923C0210923D0210923E0260E084E0F1
:1028A00090E00E94083260E082E290E00E940832EC
:1028B00060E085E090E00E94083260E086E090E011
:1028C0000E9408326FEF87E090E00E94083240E0FB
:1028D00050E0BA0188E090E00E941A3260E08DE09A
:1028E00090E00E94083240E050E0BA0188E190E0B8
:1028F0000E941A3260E087E190E00E94083240E0D6
:1029000050E0BA018CE190E00E941A3260E070E081
:1029100080E290E00E94263240E050E0BA0188E177
:1029200090E00E941A3240E050E0BA018FE090E05F
:102930000E941A3240E050E0BA0183E190E00C942A
:102940001A3280913A02811110923A0208958095CC
:10295000909139028923809339020895EF92FF9272
:102960000F931F93CF939091390280913802982B47
:102970009093EF0180913A02882389F0892B80930C
:10298000EF01E1EFF1E097E080E0915029F0219133
:102990002223D9F38F5FF9CF81110E94A11448E05F
:1029A00050E060E372E08FEE91E00E94F432892BF8
:1029B00009F448C088E0EFEEF1E0A0E3B2E0019056
:1029C0000D928A95E1F7E0916702F09168023097E5
:1029D000C9F10280F381E02D8FEE91E0099580919D
:1029E0005C0282FF2FC080FF04C085E692E00E9457
:1029F00047080FEE11E0C8E08FE5E82E82E0F82EE0
:102A000080915C0280FF0CC0F80180811F928F933F
:102A1000FF92EF920E94E0080F900F900F900F909E
:102A2000C1500F5F1F4FC111EBCF80915C0280FF3F
:102A300009C08DE592E0CF911F910F91FF90EF902B
:102A40000C944708CF911F910F91FF90EF9008953C
:102A500020912F028095822380932F02982F9770C8
:102A600099F430E0482F082E000C550B2417350739
:102A700059F090914C0292FD07C0859585958595FA
:102A80000E948C3010922F020895CF93DF93C09153
:102A90004C02C2FB992790F9981719F1D82F80FBA7
:102AA000C2F9C0934C0260914B0284E090E00E9416
:102AB00008326C2F82E290E00E94083282E00E948D
:102AC000281580915C0280FF0CC01F92DF9388E480
:102AD00092E09F938F930E94E0080F900F900F90C9
:102AE0000F90DF91CF91089580912E029091FD017A
:102AF000891719F08F5F8770FBCF08950F931F938D
:102B0000CF93DF938091FC0182958F7009F05DC0B7
:102B10008091F901882309F458C080912E02109108
:102B2000FD016091F7017091F801C091FA01D09117
:102B3000FB0191E06F3F09F090E0292F06E081173B
:102B400009F443C0209721F07F3F21F030E003C01B
:102B500031E001C0322F90E030FD34C0089FF00119
:102B6000099FF00D1124DF01A250BE4F11963C9138
:102B70001197371327C03C91361324C012963C910D
:102B8000129731111FC013964D915C9114974C1BF5
:102B90005D0B483C5105B0F48091FC018F70806161
:102BA0008093FC01ED5FFD4F80818F708061808399
:102BB00087EF91E00E949109DF91CF911F910F91D2
:102BC0000C94741501968770BACFDF91CF911F9145
:102BD0000F910895CF93DF93D82FC92F0E94D22F42
:102BE000EC2FF0E095E0899FE00DF11D1124EE0F30
:102BF000FF1FEE0FFF1FED0FF11DEE0FFF1FE05E39
:102C0000FD4F859194910E948B12DF91CF91089591
:102C10009F92AF92BF92CF92DF92EF92FF920F936B
:102C20001F93CF93DF93CDB7DEB761970FB6F894BC
:102C3000DEBF0FBECDBF8C0185E0F801DE011D9621
:102C400001900D928A95E1F7F801E2809091F701E9
:102C50006091F8014091FA015091FB014115510535
:102C600031F06F3F31F481E09F3F19F403C081E000
:102C700001C080E0F82FF1709F2E80FD1AC1F8018D
:102C800030812181C380D48087EFA82E81E0B82EC7
:102C9000F090F901F601E41BF50BFF2009F4C6C022
:102CA0008091FC01E83CF10508F091C0482F407F7D
:102CB00009F050C0621311C093130FC0FE2CE11035
:102CC0000CC08F7080618093FC01C5010E94910946
:102CD0008091FC01F801858329C1CD2831F02F3F77
:102CE00031F481E03F3F19F403C081E001C080E08E
:102CF00080FD03C081E08E2502C080E090E0F82FC7
:102D0000F170FF2E80FF1CC080912E024091FD01CA
:102D100056E0841709F4E8C090E0589FF001599FED
:102D2000F00D1124E250FE4F6181261306C0608130
:102D3000631303C06281E61203C001968770E9CF76
:102D4000FE2CEE2009F4F2C08091FC01816080939A
:102D5000FC0149C0621306C0931304C0E11002C015
:102D6000F80186C0C8010E94DC30882351F1EE20B2
:102D700041F12091FC01822F82958F7090E00297A3
:102D800074F08091F7019091F80198878F831986EC
:102D9000DB86CA862C87CE0107960E94910986E0C1
:102DA000F801A7EFB1E001900D928A95E1F70E943A
:102DB0007E150AC06217C9F0C8010E94DC3081117B
:102DC0001EC0C8010E949109FF24F394AFC0482F90
:102DD000407F81F787EF91E00E94910986E0F5013D
:102DE00011928A95E9F7F12CA1C09313E5CFE11078
:102DF000E3CFF8018583C8010E94910954C0EE20F9
:102E000001F32091FC01822F82958F7090E0029750
:102E100034F28091F7019091F8019A8389831B82A3
:102E2000DD82CC822E83CE010196B7CFE83CF1053E
:102E3000D0F5FE2CEE2029F2621327C0931325C093
:102E40002091FC0120FD18C0822F82958F70482FA1
:102E500050E04115510581F0F80125834F305105AF
:102E600041F08F5F982F9295907F822F8F70892BE2
:102E70008583C8010E94910986E0F801A7EFB1E0BF
:102E800001900D928A95E1F751C0C8010E94DC3093
:102E9000811185CF8091FC0181608093FC01C80184
:102EA0000E94910943C086E0F50111928A95E9F7E5
:102EB0003DC0EE2009F485CFC8010E94DC30F82E19
:102EC000882309F47ECF86E0F801A7EFB1E00190F6
:102ED0000D928A95E1F78091F7019091F8010E9497
:102EE000EA150E947E1522C03D872E878D859E851E
:102EF0000E94EA15292F22952F70223028F49F7006
:102F000039F0811105C00BC0243028F49F7049F4BA
:102F1000805E883020F0C8010E9491099F2CF92C16
:102F200005C0F8019581907F99F7F9CF8F2D6196B3
:102F30000FB6F894DEBF0FBECDBFDF91CF911F91CA
:102F40000F91FF90EF90DF90CF90BF90AF909F9048
:102F50000895CF93DF93CDB7DEB763970FB6F8949C
:102F6000DEBF0FBECDBF84B7877F84BF0FB6F89496
:102F7000A895809160008861809360001092600045
:102F80000FBE90E080E80FB6F894809361009093B4
:102F900061000FBE85B7806885BF85B7806885BF33
:102FA0008EE79CE19093ED018093EC010E94AD26A9
:102FB0000E94CC268091E20084608093E2007894A5
:102FC000809183028823A1F01091E9001F709091F5
:102FD000EC00892F817090FD80E8182B1092E90099
:102FE0008091E80083FD0E949B231F701093E900ED
:102FF00082E084BD93E095BD9AEF97BD80936E000B
:1030000002E511E057E5E52E51E0F52ED8018D914E
:103010008D018F3F11F00E94AC11E016F106B1F75F
:1030200007E511E04BE5E42E41E0F42EF801819133
:103030008F018F3F11F00E94AC11E016F106B1F73D
:1030400085E0E0E5F2E0DF01282F1D922A95E9F7FF
:10305000E2E4F2E0DF011D928A95E9F780E090E07A
:103060000E940232893E9E4F11F00E94361482E087
:1030700090E00E94F43180935C020E9425149093AA
:103080004C0280934B020E94C311EFEFF6E721E060
:10309000E150F0402040E1F700C000000E94C31161
:1030A0008091500280FF08C06FEF7FEF80E090E0DA
:1030B0000E9426320E948B1E83E090E00E94F43131
:1030C000682F70E080E090E00E94D230279A2F981D
:1030D0008AE08093800089E1809381008FEF9FEFE9
:1030E00090938700809386000E947B280E947B2813
:1030F00080914D028111E0C080915C0280FF08C088
:1031000089EB93E09F938F930E94E0080F900F90BC
:1031100080915C0280FF08C083EA93E09F938F93C5
:103120000E94E0080F900F9080E090E00E94023231
:10313000893E9E4F81F080915C0280FF08C08BE742
:1031400093E09F938F930E94E0080F900F900E944E
:1031500036140E941C2D88E090E00E94FC316093A0
:10316000B6027093B7028093B8029093B9026E7F53
:10317000D1F480915C0280FF08C082E393E09F93CA
:103180008F930E94E0080F900F900E941C2D88E002
:1031900090E00E94FC316093B6027093B702809376
:1031A000B8029093B9020E948A2C80915C0280FF41
:1031B00008C089E193E09F938F930E94E0080F90ED
:1031C0000F9080915C0280FF0FC08091B6028170E9
:1031D0001F928F938CEF92E09F938F930E94E00851
:1031E0000F900F900F900F9080915C0280FF0FC0A6
:1031F0008091B60286951F928F9381EE92E09F9305
:103200008F930E94E0080F900F900F900F90809185
:103210005C0280FF0EC08091B7021F928F9387ECF3
:1032200092E09F938F930E94E0080F900F900F9071
:103230000F9080915C0280FF0EC08091B8021F92B7
:103240008F938DEA92E09F938F930E94E0080F90F6
:103250000F900F900F9080915C0280FF0EC08091C4
:10326000B9021F928F9383E992E09F938F930E94FC
:10327000E0080F900F900F900F9080915C0280FFFC
:103280000EC08091BA021F928F9387E792E09F93BE
:103290008F930E94E0080F900F900F900F90109264
:1032A00094028091B60280FF04C060E086950E947F
:1032B000AF2C81E080934D0280E091E09093680212
:1032C0008093670225E5222E22E0322E31E5432E3F
:1032D00034E0532E80918302853009F0A2C083E44C
:1032E00094E00E94470890E4F92EEE24E39400E174
:1032F00012E180918302853009F069C080918302D8
:10330000843009F454C080E00E94B7220E94C12892
:1033100080914F02811128C0E0924F028091B60245
:10332000982F917090934E028E7F8093B602809179
:103330005C0280FF0CC01F921F9280ED93E09F9370
:103340008F930E94E0080F900F900F900F900E94B3
:10335000C128BFEFE0E7F2E0B150E040F040E1F714
:1033600000C000000E94F22810926B0228E130E0B9
:103370000FB6F894A895209360000FBEF0926000FD
:1033800083B7817F846083BF83B7816083BF789474
:10339000889583B78E7F83BF0FB6F894A8958091E8
:1033A0006000886180936000109260000FBE809181
:1033B0008202882309F49DCF0E94C311E0E5F2E068
:1033C000819181117CC22E163F06D1F792CF0E94C7
:1033D000FC300E947B280E945F1F10924F02809158
:1033E0004E028823E1F08091B60281608093B6029C
:1033F00080915C0280FF0DC01F9281E08F938AE074
:1034000094E09F938F930E94E0080F900F900F908D
:103410000F908091B60260E086950E94AF2C0E94CA
:10342000D0280E94C311882359F08FB7F894409197
:103430006C0250916D0260916E0270916F028FBFAD
:10344000A5E56A2EA2E07A2EB0E5CB2EB2E0DB2E07
:1034500000E010E089E4A82E84E0B82E0B8BD601A2
:10346000ED916D01EA8BD3018D913D01E827E98B48
:10347000E11116C00F5F1F4F0530110579F78FEF6F
:103480008C878D871E860E94E41E8160782F988B22
:103490008F874C855D856E8588890E94E9085BC0B1
:1034A00080915C0281FD04C080E0FF24F39435C06C
:1034B00086E594E00E944708F0E58F2EF2E09F2E0B
:1034C000E12CF12CFF92EF925F924F920E94E00864
:1034D0008EE494E00E944708F40181914F010E941C
:1034E00057111F928F93BF92AF920E94E00887E41A
:1034F00094E00E944708FFEFEF1AFF0A0FB6F89416
:10350000DEBF0FBECDBF35E0E316F104D9F6CCCF58
:103510008F5FFF0C843009F4ADCF99899F21C1F3EF
:103520008F834B8948879A899F2181E009F480E045
:1035300089870E94E41E8160782F9B878A874F814C
:10354000588569858B850E94E908F801EB5AFD4F83
:103550008081F826F08280919402882309F493C038
:1035600080919302E091B602E695E81BE0938F020A
:10357000823059F4F0E0ED58FB4FE4910E2F10E04B
:10358000EBE4EE2EEBE2FE2E59C0863059F4F0E06B
:10359000E059FB4FE4910E2F10E07BE3E72E7BE236
:1035A000F72E4CC0893061F4E695F0E0E359FB4F0B
:1035B000E4910E2F10E066EAE62E6AE2F62E3EC097
:1035C0008F3061F4E695F0E0E659FB4FE4910E2F61
:1035D00010E059E3E52E5AE2F52E30C0853159F45A
:1035E000F0E0E959FB4FE4910E2F10E04BEEE42E92
:1035F00049E2F42E23C08831A1F0833249F4E5E694
:10360000F4E00591149131EEE32E3AE2F32E16C068
:10361000843271F404EF11E028E2E22E29E2F22E66
:103620000DC008E210E092E6E92E99E2F92E06C0FC
:1036300000ED17E088E5E82E88E2F82E80919002F0
:10364000882361F0109290020E94E41E90938E02F3
:1036500080938D0210929202109291020E94E41EB9
:10366000E0918D02F0918E028E1B9F0B8F3F9F4742
:1036700050F40E0F1F1F10938E0200938D028DE8E1
:1036800092E0F701099586E0E3ECF2E0DE011196A5
:1036900001900D928A95E1F7E090C502F090C60284
:1036A0000091C7021091C8021092C5021092C60282
:1036B0001092C7021092C802E11003C0FF2009F463
:1036C0005DC08091C1029091C2020E94D51EAC01E2
:1036D0009091BE02992339F02091100130E0241717
:1036E000350758F04BC020911101FAE02F9F90014F
:1036F00011242417350718F041C09F3F19F09F5F30
:103700009093BE02EE2061F00E941D2F1E1414F053
:103710009FEF01C091E0899F802D11248093C50205
:10372000FF2061F00E941D2F1F1414F09FEF01C0B5
:1037300091E0899F802D11248093C6023091C502AB
:103740003323E1F02091C6022223C1F045EB34037C
:10375000C0011124992319F09093C50203C081E0A0
:103760008093C50235EB2303C0011124992319F07E
:103770009093C60203C081E08093C602011103C08A
:10378000112309F451C08091BF029091C0020E94A0
:10379000D51E9C019091BC02992309F4A6C0213545
:1037A000310508F441C09F3F19F09F5F9093BC0220
:1037B000002361F00E94E42E101614F09FEF01C068
:1037C00091E0899F802D11248093C702112361F01D
:1037D0000E94E42E111614F09FEF01C091E0899F22
:1037E000802D11248093C8023091C7023323E1F069
:1037F0002091C8022223C1F045EB3403C0011124FB
:10380000992319F09093C70203C081E08093C70207
:1038100035EB2303C0011124992319F09093C802BA
:1038200003C081E08093C8028091C50281110BC062
:103830008091C602811107C08091C702811103C027
:103840008091C80281110E94C12DEB82FC820D8300
:103850001E8386E0FE013196A3ECB2E001900D924A
:103860008A95E1F70E945F1F182F80915A0218175E
:1038700009F430CD10935A0280915C0282FF2ACD68
:1038800080FF04C08EE794E00E94470880915C02AC
:1038900080FF0CC01F921F9389E794E09F938F9342
:1038A0000E94E0080F900F900F900F9080915C02A3
:1038B00080FF10CD87E794E00E9447080BCD09BD3B
:1038C00019BD09B400FEFDCF8091D8008F7D809393
:1038D000D8008091E00082608093E0008091E00059
:1038E00081FDFCCF0E94FC3004CD2B30310508F067
:1038F0005CCF9ACF08958091780208959FB7F8948D
:10390000109274029FBF90918302943009F057C0C7
:103910009091E9009F703091EC00232F217030FDD1
:1039200020E8922B23E02093E9002091EB0020FF78
:1039300043C02091EE0027FF3FC020917302222355
:1039400021F02091E80025FF37C01092730226E095
:103950003091E80035FD15C030918302343061F5B7
:103960003091EB0035FD28C0215021F481E0809397
:10397000730222C0EFE9FFE03197F1F700C00000C9
:10398000E7CF8093F1008091E80085FD0AC0809127
:10399000E80080FFFCCF8091E8008E778093E800FC
:1039A00006C08FB7F89421E0209374028FBF9F70F8
:1039B0009093E90080E008959F709093E9008FEF65
:1039C00008958093700270937202609371028091E7
:1039D0008302843001F582E08093E9008FEF9091BB
:1039E000E800815095FD06C095ED9A95F1F700002D
:1039F0008111F5CF8091E80085FF0DC040E050E0D7
:103A000063E070E080E792E00E946F238091E8001D
:103A10008E778093E8000895BC0184E00C94E11C4B
:103A2000BC0183E00C94E11C22E02093E9002FEF1D
:103A30003091E800215035FD06C035ED3A95F1F79B
:103A400000002111F5CF2091E80025FF0BC040E0D8
:103A500050E066E070E00E946F238091E8008E776E
:103A60008093E8000895CF93DF9321E02093E9004D
:103A70002FEF3091E800215035FD06C035ED3A9525
:103A8000F1F700002111F5CF2091E80025FF14C0C7
:103A9000EC0140E050E068E070E00E946F2380910C
:103AA000E8008E778093E80088E0FE01A9E7B2E0A5
:103AB00001900D928A95E1F7DF91CF910895809161
:103AC0000C011F928F9380910D011F928F93809113
:103AD0000E011F928F9380910F011F928F938091FF
:103AE00010011F928F93809111011F928F9380EA92
:103AF00099E09F938F930E94E0088DB79EB70E9632
:103B00000FB6F8949EBF0FBE8DBF0895CF93C82FF8
:103B10001F928F9384E39BE09F938F930E94E00812
:103B200081E090E0A0E0B0E0BC01CD0104C0660FF0
:103B3000771F881F991FCA95D2F70E94D2300F9025
:103B40000F900F900F90CF910C94FC302091E400D7
:103B50003091E50095E64091EC00842F817040FFA4
:103B600023C08091E80080FD1DC0809183028823DE
:103B700099F0853099F08091EB0085FD11C040915E
:103B8000E4005091E5002417350729F3915011F016
:103B90009A01E1CF84E0089582E0089583E00895DA
:103BA00081E0089580E008954091E80042FFDDCF74
:103BB00008958091850287FF11C08091E80082FD01
:103BC00005C0809183028111F8CF11C08091E80077
:103BD0008B770BC080918302882349F08091E800A5
:103BE00080FFF8CF8091E8008E778093E8000895F9
:103BF000982F973068F59093E900981739F07091F5
:103C0000EC002091ED005091F00003C0242F762F9E
:103C100050E021FD02C09F5FECCF3091EB003E7F72
:103C20003093EB003091ED003D7F3093ED0030910B
:103C3000EB0031603093EB007093EC002093ED00CB
:103C40005093F0002091EE0027FDE5CF80E008952D
:103C50008F708093E90081E0089520918B0230916C
:103C60008C022617370748F06115710539F4209149
:103C7000E8002E772093E80001C0B901FC0120E0A4
:103C80006115710579F1809183028823F1F1853006
:103C9000F1F18091E80083FD3CC08091E80082FD55
:103CA0002EC08091E80080FFEBCF2091F30080913F
:103CB000F20090E0922B6115710551F0883091056A
:103CC00038F421912093F100615071090196F3CFEE
:103CD00021E0089709F020E08091E8008E7780933A
:103CE000E800CECF2111CFCF0AC080918302882374
:103CF00061F0853061F08091E80083FD0AC0809119
:103D0000E80082FFF2CF80E0089582E0089583E02A
:103D1000089581E0089581E08093E00080E280933F
:103D2000D8001092C9008FE19EE40197F1F700C01E
:103D3000000087E090EBDC018093D8029093D902D9
:103D4000A093DA02B093DB029CE088E10FB6F8940E
:103D5000A895809360000FBE90936000FFCF789489
:103D60001F920F920FB60F9211248F939F93AF93D0
:103D7000BF9380916C0290916D02A0916E02B09100
:103D80006F020196A11DB11D80936C0290936D028C
:103D9000A0936E02B0936F02BF91AF919F918F91EC
:103DA0000F900FBE0F901F9018959C014FB7F8947D
:103DB00080916C0290916D02A0916E02B0916F02A1
:103DC0004FBF821B930B08952FB7F89480916C021C
:103DD00090916D02A0916E02B0916F022FBF089575
:103DE0001F920F920FB60F9211248F939F93AF9350
:103DF000BF9380916B02811113C080916C029091EE
:103E00006D02A0916E02B0916F024196A11DB11D8D
:103E100080936C0290936D02A0936E02B0936F0238
:103E2000BF91AF919F918F910F900FBE0F901F90F8
:103E300018959C01FC0132969FEF80E04191461756
:103E400089F09F3F19F4411101C0982F8F5F863090
:103E5000A9F79F3F39F0F901E90FF11D97FDFA9598
:103E60006283089508952091690230916A022817AB
:103E7000390771F090936A0280936902E0916702BA
:103E8000F0916802309721F00084F185E02D0994CB
:103E9000089520916502309166022817390771F064
:103EA0009093660280936502E0916702F091680248
:103EB000309721F00680F781E02D09940895E09174
:103EC0006702F0916802309721F00190F081E02DB7
:103ED000099480E00895EF92FF920F93CF93DF93C0
:103EE000C42FD22FFC0182818823D1F04093640239
:103EF0000E94E41E909363028093620280E28C0F22
:103F0000883008F06DC0C77081E001C0880FCA9585
:103F1000EAF7DF91CF910F91FF90EF900C940E3163
:103F20008091640248134BC08091620290916302B9
:103F30000E94D51E883C910508F041C0CD17C9F0FC
:103F400080E28C0F883040F4C77081E001C0880F98
:103F5000CA95EAF70E94073180E28D0F883048F455
:103F600081E09D2F977001C0880F9A95EAF70E9413
:103F70000E31093319F0E12CF12C03C080E5E82E55
:103F8000F12C802F0E945031E114F10451F08FE99F
:103F90009FE00197F1F700C0000091E0E91AF108F5
:103FA000F3CF802F0E94183180E28D0F8830C0F44B
:103FB000D77081E001C0880FDA95EAF70AC080E285
:103FC0008C0F883068F4C77081E001C0880FCA95F3
:103FD000EAF7DF91CF910F91FF90EF900C940731AA
:103FE000DF91CF910F91FF90EF900895883220F5E7
:103FF0008E3108F068C08B3091F1C0F4873009F041
:10400000BEC081E08093110184E1809310018AE0B9
:1040100080930F018EE180930E0188E080930D0163
:1040200088E280930C0182E09BE0C6C0833109F4F2
:1040300043C0843169F1A3C08F3409F49EC028F4D1
:10404000893231F1883359F09AC0813531F008F462
:10405000D4C0823509F4A7C092C08FEFA5C084E216
:104060009BE00E9447080E945F1D1F9281E08F9392
:104070001F9288E08F938DE19AE09F938F930E9427
:10408000E0080F900F900F900F900F900F9096C038
:1040900081E29BE00E94470880916102882309F435
:1040A000AAC0109261021092600210925F021092F8
:1040B0005E0210925D02B1C083E19BE00E9447085E
:1040C0000E945F1D7BC08D5180936102833031F16E
:1040D00070F48130D1F0823009F03FC080E191E08E
:1040E0009093600280935F0288E691E01FC0853064
:1040F00059F108F1863089F58CE091E090936002E7
:1041000080935F0283EA91E011C081E191E0909396
:10411000600280935F028FE591E008C08FE091E03C
:104120009093600280935F0284E791E090935E0237
:1041300080935D0218C08EE091E0909360028093BE
:104140005F0281E891E0F2CF8DE091E09093600210
:1041500080935F0280E991E0E9CF1092610280E1F3
:104160009BE00E94470880916102882309F455C0B2
:104170001F928F938CE09BE00DC08AE015C08FEFFB
:104180009AE01AC097FF47C0108280811F928F93D8
:1041900089EF9AE09F938F930E94E0080F900F9011
:1041A0000F900F900BC081E0E0915F02F0916002F0
:1041B000309729F586EF9AE00E9447082091610226
:1041C000222359F180915D0290915E02009711F4D3
:1041D0008BE591E09F938F931F922F938DEE9AE042
:1041E0009F938F930E94E0080F900F900F900F9075
:1041F0000F900F9016C080E0089586EFD5CF2081F4
:10420000082E000C990B820F911D8F3F910509F02C
:104210000CF4B8CF8FEF8083B8CF89EE9AE00E947C
:10422000470881E00895CF92DF92EF92FF92CF93FB
:10423000DF938B3109F418C108F0B0C08B3009F45A
:10424000D2C008F09AC0863009F4D0C020F485307E
:1042500009F4DEC07FC1873009F4EBC0883009F073
:1042600079C183E090E00E94F4311F928F938AEE2F
:1042700095E09F938F930E94E00882E090E00E9477
:10428000F43183FB992790F91F929F9382FB992722
:1042900090F91F929F9381FB992790F91F929F930A
:1042A000982F91701F929F931F928F9381EA95E0B0
:1042B0009F938F930E94E0080E94251487FB22277A
:1042C00020F91F922F9386FB222720F91F922F930C
:1042D00085FB222720F91F922F9384FB222720F9A8
:1042E0001F922F9383FB222720F91F922F9382FB8B
:1042F000222720F91F922F9391FB222720F91F924A
:104300002F93292F21701F922F9381FB222720F9B1
:104310001F922F93282F21701F922F939F938F937B
:104320008CEB94E09F938F930E94E0088DB79EB72B
:1043300088960FB6F8949EBF0FBE8DBF86E090E0C2
:104340000E94F431982F9695969596951F929F937B
:10435000982F91701F929F931F928F9389E894E0FA
:104360009F938F930E94E0088DB79EB708960FB673
:10437000F8949EBF0FBE8DBFEBC0803109F49CC086
:1043800020F48E3009F484C0E5C0863109F4B1C050
:10439000893109F0DFC081ED97E0A8C08A32E1F0F1
:1043A00060F4873209F4D1C028F48E3108F4D2C009
:1043B0008D51CCC0893261F1CDC0833448F48A3349
:1043C00008F0C1C0853309F4C0C0883361F0C2C0B1
:1043D000833409F4BAC0BEC08FE899E00E94470850
:1043E0000E943614B5C087E096E080C080915C02E0
:1043F000817F8E7F80935C028AEA97E00E94470863
:104400008BE899E00E94470881E080935B02A0C09E
:104410008FE699E00E9447080E94FC309FEF24E35A
:104420008CE0915020408040E1F700C000000E94E5
:104430008B1E80915C02C82FC095C170C0FB80F9B3
:1044400080935C02CC2329F083E699E00E94470820
:1044500086C086E599E00E94470880915C02897FCA
:10446000877F80935C0274C090915C0291FBCC27A3
:10447000C0F981E0C827892FC0FB81F980935C02D5
:10448000CC2319F089E499E027C08BE399E02EC092
:1044900090915C0292FBCC27C0F981E0C827892F5C
:1044A000C0FB82F980935C02CC2319F08CE299E086
:1044B00013C08CE199E01AC090915C0293FBCC2769
:1044C000C0F981E0C827892FC0FB83F980935C0283
:1044D000CC2351F080E199E00E94470880915C0272
:1044E000816080935C023BC083E099E00E944708B2
:1044F0002FC08FB7F894C0906C02D0906D02E090FE
:104500006E02F0906F028FBFD0917702C0911201BE
:104510000E945F1FFF92EF92DF92CF921F92DF9374
:104520001F92CF931F928F9386E998E09F938F936A
:104530000E94E0088DB79EB70C960FB6F8949EBF08
:104540000FBE8DBF05C0895301C080E00E94861D4B
:10455000C1E005C081E099E00E944708C0E08C2FCF
:10456000DF91CF91FF90EF90DF90CF9008958F92E1
:104570009F92AF92BF92CF92DF92EF92FF920F93F2
:104580001F93CF93DF93843048F4811108C090913A
:104590008000977F909380002F9806C083E09091D1
:1045A0008000986090938000A0918600B091870071
:1045B000282F30E00E94BE3223E030E040E050E09F
:1045C0000E948E320027122F232F342F012F122FFB
:1045D000232F332780918600909187006CE070E054
:1045E0000E9466326017710730F0C80169E070E020
:1045F0000E9466325EC08091860090918700E090B4
:104600008600F0908700E0918600F0918700C6E078
:10461000D0E0BE010E946632060F171F211D311D1A
:104620004801590185E0880C991CAA1CBB1C8A957D
:10463000D1F7C701BE010E9466326F01E12CF12C57
:10464000A7019601260F371F411D511DC501B40159
:104650000E948E3269017A01E0918600F091870014
:10466000CA01B9010E943C329B01AC01DF010E94EA
:10467000D4329B01AC01C701B6010E943C32DC017F
:10468000CB012FE0B695A795979587952A95D1F7F9
:10469000009186001091870020E030E0081719078C
:1046A0002A073B0728F46091860070918700CB01B0
:1046B000BC0170938D0060938C00DF91CF911F91AE
:1046C0000F91FF90EF90DF90CF90BF90AF909F90B1
:1046D0008F900895682F86E090E00C940832EF9256
:1046E000FF920F931F93CF93DF937C018B010E9466
:1046F000A61D811119C0E70101151105A1F08091D6
:10470000E80085FD0AC08091E8008E778093E8007C
:104710000E94A61D882381F307C089918093F10030
:1047200001501109E9CF80E0DF91CF911F910F91E6
:10473000FF90EF9008951F93CF93DF93CDB7DEB72F
:10474000AA970FB6F894DEBF0FBECDBFE5E8F2E042
:104750008091F100819342E0ED38F407C9F7809130
:104760008602833009F461C030F4813071F0823008
:1047700009F49BC0B2C08A3009F487C08B3009F4B9
:104780006CC0893009F0A9C020C080918502813AAF
:1047900009F0A3C08091E800877F8093E8008091B2
:1047A000890290918A02892B21F468E089E792E0DE
:1047B00003C060E080E090E070E00E942D1E8091D8
:1047C000E8008B778093E80088C080918502813271
:1047D00009F083C08091890290918A02029708F0C3
:1047E0007CC08091E800877F8093E8008091E8009A
:1047F00082FD05C0809183028111F8CF6EC02091A7
:10480000F3008091F20090E0922B029731F48091B6
:10481000F100813011F0863021F48091F100809315
:1048200078028091E8008B7754C080918502813AAC
:1048300009F053C08091890290918A02892B09F076
:104840004CC08091E800877F8093E8008091E80069
:1048500080FFFCCF8091120137C0809185028132A8
:10486000E1F58091890290918A02892BB1F58091BE
:10487000E800877F8093E8000E94D91D809187021D
:10488000809312010E94FC3028C080918502813201
:1048900021F58091E800877F8093E8000E94D91D70
:1048A000809188028093770218C080918502813AB6
:1048B000A1F48091E800877F8093E8008091E80070
:1048C00080FFFCCF809177028093F1008091E80017
:1048D0008E778093E8000E94D91D8091E80083FFC5
:1048E000DAC18091850290918602492F50E04A30CA
:1048F000510508F0D0C1FA01EE59FF4F0C94B032C7
:10490000803821F0823809F0C6C108C08091810248
:1049100090918202992389F082600FC08091890270
:104920008F70873008F0B7C18093E9008091EB0069
:1049300085FB882780F91092E9009091E800977F25
:104940009093E8008093F1001092F10070C1282F3D
:104950002D7F09F0A0C1882319F0823061F09BC13E
:1049600080918702813009F096C1933009F080E090
:10497000809382022EC08091870281112AC080918B
:1049800089028F702FEF280F263008F084C18093A2
:10499000E9002091EB0020FF1CC0933021F48091AE
:1049A000EB00806214C09091EB0090619093EB005B
:1049B00021E030E0A90102C0440F551F8A95E2F7BB
:1049C0004093EA001092EA008091EB0088608093A7
:1049D000EB001092E9008091E800877F8093E80067
:1049E0000E94D91D58C1811156C1109187021F77AD
:1049F0008091E3008078812B8093E3008091E80030
:104A0000877F8093E8000E94D91D8091E80080FF95
:104A1000FCCF8091E30080688093E300111102C015
:104A200082E001C083E08093830235C180588230E8
:104A300008F031C120918702309188022C3D53E06B
:104A4000350779F583E08A838AE289834FB7F89442
:104A5000DE01139620E03EE051E2E32FF0E05093B8
:104A60005700E49120FF03C0E295EF703F5FEF70C5
:104A70008E2F90E0EA3010F0C79601C0C0968D935B
:104A80009D932F5F243149F74FBF8091E800877FC6
:104A90008093E8006AE270E0CE0101960E942D1E2C
:104AA000B5C08091890290918A02432F55274330E7
:104AB0005105A9F068F44130510509F4FBC04230BA
:104AC000510509F0E8C08BE590E0EAE2FCE04BC05C
:104AD0004132510529F14232510589F1DCC0C90149
:104AE000992781309105A1F058F0029709F0D3C0C1
:104AF000E7E9FCE0E4918E2F90E0E7E9FCE030C0CC
:104B0000E9ECFCE0E4918E2F90E0E9ECFCE028C0B9
:104B1000E9EAFCE0E4918E2F90E0E9EAFCE020C0B5
:104B20008330910508F0B7C0880F991FFC01EF533F
:104B3000FE4F0190F081E02D89E090E014C08330B9
:104B4000910508F0A8C0FC01EE0FFF1FE554FE4FD1
:104B50000190F081E02DDC01A854BE4F8C9190E0D3
:104B6000009709F498C02091E800277F2093E8007F
:104B700020918B0230918C028217930708F49C01DC
:104B800040E02115310589F180918302882309F4E1
:104B90003DC08530D9F18091E80083FD37C0809118
:104BA000E80082FD2FC08091E80080FFEACF4091AD
:104BB000F3008091F20090E0942B2115310559F01B
:104BC0008830910540F444914093F1003196215092
:104BD00031090196F2CF41E0089709F040E0809159
:104BE000E8008E778093E800CCCF4111CDCF0AC08A
:104BF00080918302882351F0853041F08091E80054
:104C000083FD04C08091E80082FFF2CF8091E8002C
:104C10008B778093E8003FC08038E9F58091E80009
:104C2000877F8093E800809184028093F1008091D7
:104C3000E8008E77D3CE81112EC0809187029091AB
:104C40008802992702973CF58091E800877F80933E
:104C5000E80010918702109384020E94D91D11115F
:104C600006C08091E30087FD02C081E001C084E0BE
:104C70008093830242E061EC81E00E94F81D42E2F1
:104C800061EC82E00E94F81D42E261EC83E00E9448
:104C9000F81D809183028091E80083FF10C080910D
:104CA000E800877F8093E8008091EB00806280932A
:104CB000EB0005C082E190E0E5E8FCE054CFAA9665
:104CC0000FB6F894DEBF0FBECDBFDF91CF911F911D
:104CD00008951F920F920FB60F9211242F933F93B6
:104CE0004F935F936F937F938F939F93AF93BF93F4
:104CF000CF93DF93EF93FF93C091E900CF70809142
:104D0000EC00D82FD17080FDD0E81092E90080919E
:104D1000F000877F8093F00078940E949B2310928C
:104D2000E9008091F00088608093F000CD2BCF7077
:104D3000C093E900FF91EF91DF91CF91BF91AF91C7
:104D40009F918F917F916F915F914F913F912F91A3
:104D50000F900FBE0F901F901895E8EDF0E0808146
:104D60008E7F80831092E2001092DA001092E100B0
:104D7000A0EEB0E08C9181608C9380818F778083EE
:104D800019BCA7EDB0E08C918E7F8C9380818F7ED3
:104D90008083109276020895CF92DF92EF92FF9275
:104DA0000F931F93CF93DF93C8EDD0E088818F7E60
:104DB0008883E7EDF0E080818160808384E082BFBA
:104DC00081E08093760288818E7F888302EE10E0F6
:104DD000F80110821092DA0081EEC82ED12CF60173
:104DE000108288818F778883888180688883888112
:104DF0008F7D888319BC10928302109284021092D6
:104E000082021092810290EEE92EF12CF70180814E
:104E10008B7F808388818160888342E060E080E0CE
:104E20000E94F81DF60180818E7F8083F8018081C9
:104E300081608083808188608083F70180818E7F9C
:104E40008083888180618883DF91CF911F910F914A
:104E5000FF90EF90DF90CF9008951F920F920FB6C2
:104E60000F9211242F933F934F935F936F937F93F0
:104E70008F939F93AF93BF93EF93FF938091E10044
:104E800082FF49C08091E20082FF45C08091E1002D
:104E90008B7F8093E100209175022F5F822F62E368
:104EA0000E944C32992319F02093750234C010925D
:104EB000750280917402882371F18091830284309D
:104EC00041F58091E9008F702091EC00922F917054
:104ED00020FD90E8892B93E09093E9009091EB00FE
:104EE00090FF14C09091EE0097FF10C09091E800E1
:104EF00095FF03C01092F100F9CF9091E80090FF68
:104F000005C09091E8009E779093E8008F708093A1
:104F1000E900109274028091DA0080FF32C0809123
:104F2000D80080FF2EC08091DA008E7F8093DA0057
:104F30008091D90080FF1CC080E189BD82E189BDDC
:104F400009B400FEFDCF81E08093830286E19CE0FE
:104F50000E94470880917602811113C00E94AD26FD
:104F60000E94CC268091E20084608093E20009C018
:104F700019BC109283028AE19CE00E9447081092BB
:104F800076028091E10080FF1BC08091E20080FFEB
:104F900017C08091E2008E7F8093E2008091E20052
:104FA00080618093E2008091D80080628093D80075
:104FB00019BC85E0809383028EE19CE00E94470843
:104FC0008091E10084FF34C08091E20084FF30C012
:104FD00080E189BD82E189BD09B400FEFDCF8091E9
:104FE000D8008F7D8093D8008091E1008F7E8093E0
:104FF000E1008091E2008F7E8093E2008091E200E8
:1050000081608093E20080918402882311F084E023
:1050100007C08091E30087FD02C081E001C083E00A
:105020008093830282E29CE00E9447088091830281
:105030008091E10083FF2BC08091E20083FF27C0B5
:105040008091E100877F8093E10082E0809383027A
:10505000109284028091E1008E7F8093E100809124
:10506000E2008E7F8093E2008091E2008061809375
:10507000E20042E060E080E00E94F81D8091F000D4
:1050800088608093F00086E29CE00E944708FF91D0
:10509000EF91BF91AF919F918F917F916F915F91B0
:1050A0004F913F912F910F900FBE0F901F90189529
:1050B00008958091BA02882319F081508093BA0232
:1050C0006091B6027091B7028091B8029091B902D6
:1050D0000C949D2C8091BA02833018F48F5F8093DA
:1050E000BA026091B6027091B7028091B8029091B5
:1050F000B9020C949D2C80E090E00E940232893E1F
:105100009E4F51F00E9436148091BB0284708961D9
:105110008093BB020E946A2386E090E00E94F431F3
:105120008093BB02282F26952695269530E02430C3
:10513000310524F0877088618093BB028091BB02A7
:1051400080FF04C086958695869501C080E00C940A
:10515000B7229091B60290FF04C09695981740F040
:1051600003C0811105C090E0961710F40C94122D25
:1051700061E00C94AF2C882311F0FA0101C0FB010F
:1051800009941092940280915C0280FF08C08EE521
:105190009DE09F938F930E94E0080F900F900895D9
:1051A0006091B602669570E04BE050E083E191E0DB
:1051B0000E94E732892B19F481E0809394020E94C7
:1051C000E41E90938E0280938D0280915C0280FF9A
:1051D00008C085E49DE09F938F930E94E0080F90A4
:1051E0000F9008958091B60280FF0AC06A9A8EB12E
:1051F0008B7F9EB194602FB7F894E8E9F2E00BC082
:10520000E8E9F2E0118210821282339632E0E63B46
:10521000F307C1F7EBCF32E0E63BF30789F03191BA
:1052200048E09EB9000000C037FF8EB9330F000080
:1052300000C000C000C08EB900C04A9591F7EBCF06
:105240002FBF8FE594E00197F1F700C000000895AB
:10525000EF92FF920F931F93CF93DF938C01C8E9D6
:10526000D2E0E12CF12CF8018481F5E0EF16F10495
:105270001CF4882339F002C0811104C09E014091C2
:10528000B90202C09E0140E06091B8028091B7026D
:105290000E942B2D8FEFE81AF80A23969AE0E91660
:1052A000F10409F70E94F228F801848190E0019648
:1052B000817099278483DF91CF911F910F91FF9087
:1052C000EF9008958F929F92AF92BF92CF92DF920C
:1052D000EF92FF920F931F93CF93DF93EC014C81DA
:1052E000042F10E09801D8010E94BE329B01AC014E
:1052F0000E94D4326B017C01E0E2F0E0E01BF10B94
:10530000A5E5B0E09B01AC010E94D4324B015C01E9
:105310009F01DF010E94B6329B01AC010E94DF3287
:105320009B01AC012C0D3D1D4E1D5F1DC501B4013F
:105330000E948E32822FF22E99E2921728F093E08B
:10534000299F900111240DC025E530E0281B31096B
:10535000C901880F991F280F391F37FF02C02F5F1F
:105360003F4F35952795122F109598E9C92E92E059
:10537000D92E00E085E5E82EEF1801FD02C08E2D44
:1053800001C08F2D9601412F6091B8020E942B2DF4
:105390000F5F83E0C80ED11C0A3079F70E94F22813
:1053A0008C81811102C091E003C0803219F49FEF1B
:1053B0009093200190912001890F8C83DF91CF91F0
:1053C0001F910F91FF90EF90DF90CF90BF90AF9023
:1053D0009F908F9008950F931F93CF93DF93C8E909
:1053E000D2E0FE01118210821282339682E0E63B07
:1053F000F807C1F700E010E080919602082E000C3B
:10540000990B0817190794F080911F01082E000CC2
:10541000990B8017910754F09E014091B902609159
:10542000B8028091B7020E942B2D03C01982188206
:105430001A820F5F1F4F23960A301105E9F60E946A
:10544000F22880911E0190919602980F90939602F7
:1054500020911F01280F20931F01121614F4993078
:105460001CF0819580931E01DF91CF911F910F91C8
:105470000895BF92CF92DF92EF92FF920F931F9306
:10548000CF93DF93FC01828180FF03C0DD24DA9497
:1054900002C0DD24D39408E912E0C0E0D0E02AE0A5
:1054A000B22EF80111821082128294E0E92EF12CC2
:1054B000C12C809195028C0D8B302CF06B2D0E94AD
:1054C0005832892F02C087FD865F082E000C990B89
:1054D000C817D90791F48091B9028E9DA0018F9DC4
:1054E000500D112455954795559547959801609114
:1054F000B8028091B7020E942B2DCD0CF1E0EF1A7B
:10550000F108B9F621960D5F1F4FCA30D10549F653
:105510000E94F2288091950291E0D91206C0811173
:1055200002C089E007C0815005C090E00196BE012D
:105530000E947A3280939502DF91CF911F910F9153
:10554000FF90EF90DF90CF90BF900895EF92FF9281
:105550001F93CF93DF93EC0188E9E82E82E0F82EC9
:1055600010E08C8197014091B9026091B802810FDF
:105570000E942B2D175E83E0E80EF11C1A3F89F77D
:105580000E94F2289A818C8190FF02C08F5F01C037
:1055900081508C83DF91CF911F91FF90EF90089500
:1055A0009091B60290FF0CC0E8E9F2E0818360833D
:1055B0004283339692E0E63BF907C1F70C94F22858
:1055C00008950F931F93CF93DF9300D01F92CDB711
:1055D000DEB78C018091970281110AC09E012F5F76
:1055E0003F4F4FEF6FEF0E942B2D8A8180939702E0
:1055F000F8018481813051F028F0823061F44091CB
:1056000097020AC08091970240E007C0609197021C
:1056100040E080E003C040E080E060E00E94D02AEB
:10562000F801848190E0019663E070E00E947A3294
:1056300084830F900F900F90DF91CF911F910F9166
:105640000895CF93DF9300D01F92CDB7DEB790912E
:10565000B60290FF0AC09E012F5F3F4F0E942B2D84
:105660004B8169818A810E94D02A0F900F900F9000
:10567000DF91CF910895CF93DF93EC01E6EBF2E059
:10568000438162818C810E94212B8C818F5F8C836E
:10569000DF91CF910895CF93DF93EC01EC81F0E09F
:1056A000E958F24F4491E6EBF2E0628181810E9479
:1056B000212B8C818F5F8C83DF91CF9108952F9266
:1056C0003F924F925F926F927F928F929F92AF9292
:1056D000BF92CF92DF92EF92FF920F931F93CF93DF
:1056E000DF9300D000D0CDB7DEB7182F462E542E52
:1056F000222E9091B60290FFB4C0E92FE695AE2F0E
:10570000B0E0A953BE4F8C91809393029E7F92305C
:1057100061F49E012F5F3F4F812F0E942B2D4B8103
:1057200069818A810E94D02A62C0823019F4509027
:10573000B9025DC0863019F41091B70258C08930A3
:10574000D9F3893109F053C0E9518E2F8170382E79
:1057500081E083258C83E695F0E0E05CF24FC59014
:10576000D49088E9A82E82E0B82EE12CF12CDD241B
:105770009AE0692E712C29E1822E2DE0922EEC9C6C
:10578000C001ED9C900DFC9C900D1124B3010E9472
:105790006632012F311002C0060F01C0061B809136
:1057A0005C0280FF12C0DF92CF921F929C819F9378
:1057B0001F920F93FF92EF929F928F920E94E008A8
:1057C0000FB6F894DEBF0FBECDBF9501452D642DF9
:1057D000802F0E942B2D9FEFE91AF90A83E0A80E73
:1057E000B11C9AE0E916F10451F60E94F2281093D8
:1057F000B7024092B8025092B9022220E9F06091BB
:10580000B6027091B7028091B8029091B9020E94DD
:105810009D2C80915C0280FF24C08091B9021F9270
:105820008F938091B8021F928F938091B7021F923D
:105830008F9384EF9CE00CC080915C0280FF11C0CC
:105840001F925F921F924F921F921F938DEC9CE0CC
:105850009F938F930E94E0080FB6F894DEBF0FBEAF
:10586000CDBF0F900F900F900F90DF91CF911F91B0
:105870000F91FF90EF90DF90CF90BF90AF909F90EF
:105880008F907F906F905F904F903F902F900895F2
:10589000E6EBF2E0438128E0421B08F440E021E01F
:1058A000628181810C945F2BE6EBF2E0438128E07A
:1058B000420F08F44FEF21E0628181810C945F2B4D
:1058C000E6EBF2E0628128E0621B08F460E021E090
:1058D000438181810C945F2BE6EBF2E0628128E04A
:1058E000620F08F46FEF21E0438181810C945F2BFC
:1058F000E6EBF2E0818121E04381628188500C94E3
:105900005F2BE6EBF2E0818121E043816281885FD9
:105910000C945F2B8091B602282F269530E021153C
:10592000310519F48170826005C02532310524F0FB
:10593000817088648093B6020895CF92DF92EF92CF
:10594000FF926B017C010E948A2CB701A60188E0BE
:1059500090E0FF90EF90DF90CF900C941A329091EE
:10596000B60290FF55C09170811102C0926006C0CE
:10597000853210F0986402C0880F982B9093B6027D
:105980006623B1F06091B6027091B7028091B802BF
:105990009091B9020E949D2C80915C0280FF1BC0F7
:1059A0008091B60286951F928F938FED9FE00BC07A
:1059B00080915C0280FF0FC08091B60286951F9295
:1059C0008F9381EC9FE09F938F930E94E0080F904C
:1059D0000F900F900F906091B602669570E04BE0CB
:1059E00050E083E191E00E94E732892B19F00E9498
:1059F000C12802C00E94D02881E08093900220E05C
:105A00004091B9026091B8028091B7020C945F2B6B
:105A100008958091B6028695815009F484E261E090
:105A20000C94AF2C8091B60286958F5F853208F07A
:105A300081E061E00C94AF2CE6EBF2E083E0808340
:105A400011828FEF828383831482608171818281CE
:105A500093810C949D2CAF92BF92CF92DF92EF92E4
:105A6000FF920F931F93CF93DF93E82EF62EE90159
:105A7000E42FF0E0611106C0EF53F14FE4914E2F97
:105A80002E2F71C0062F10E0EF53F14F4491F42FE9
:105A9000C42ED12C26E0829FC00111242FEF30E0CC
:105AA000B9010E9466325BEA5603C001579F900D10
:105AB00011248E0D911D8E0D911D582F550F580FCD
:105AC000D901A01BB10BAC9DC001AD9D900DBC9D3B
:105AD000900D1124E92FF59ED0011124AB2FBB2787
:105AE0007901EA1AFB0AEC9CD001ED9CB00DFC9CFC
:105AF000B00D11245901A51AB108A09E7001A19EF4
:105B0000F00CB09EF00C1124EF2CFF242E193F094D
:105B10002C9D80012D9D100D3C9D100D1124212FD9
:105B20006230710591F048F461157105E1F0613062
:105B30007105B9F4242F4B2F16C06430710569F03C
:105B400040F06630710579F00CC0242F492FE12F09
:105B50000AC0492FEF2F2B2F06C0292FE42F412FEA
:105B600002C0292FEB2F49832883EA83DF91CF914D
:105B70001F910F91FF90EF90DF90CF90BF90AF906B
:105B8000089580915C0283FF7EC08EE99EE00E94B2
:105B900047088091C4021F928F9389E99EE09F93EA
:105BA0008F930E94E00887E99EE00E944708809159
:105BB000C502282F082E000C330B3F938F9384E9E6
:105BC0009EE09F938F930E94E00882E99EE00E94EE
:105BD00047088091C602282F082E000C330B3F93F4
:105BE0008F938FE89EE09F938F930E94E0088DE84B
:105BF0009EE00E9447088091C702282F082E000CC3
:105C0000330B3F938F938AE89EE09F938F930E947C
:105C1000E00888E89EE00E9447088091C802282F8B
:105C2000082E000C330B3F938F9385E89EE09F93E3
:105C30008F930E94E00882E89EE00E9447088091CE
:105C4000BE021F928F938FE79EE09F938F930E94D7
:105C5000E0088DE79EE00E9447088091BD021F92F8
:105C60008F938AE79EE09F938F930E94E00887E7D7
:105C70009EE00E9447088DB79EB74C960FB6F894E9
:105C80009EBF0FBE8DBF0E94E41E2091C502211150
:105C900004C02091C602222321F09093C202809377
:105CA000C1022091C702211104C02091C802222301
:105CB00021F09093C0028093BF02E0916702F091BF
:105CC0006802309749F082E08093C3020480F58136
:105CD000E02D83EC92E0099408958D3E39F4909183
:105CE000C60297FF35C01092C60259C08E3E29F4F5
:105CF0009091C6021916BCF32BC09091C5028F3E3D
:105D000029F497FF25C01092C50249C0803F19F4BD
:105D10001916CCF31DC09091C702893F29F41916BA
:105D2000BCF41092C7023BC08A3F19F497FF10C021
:105D3000F8CF8B3F39F49091C80297FF09C01092B9
:105D4000C8022DC08C3F21F49091C8021916BCF3F3
:105D50009FE0980F983080F421E030E0A90102C064
:105D6000440F551F9A95E2F7CA0180959091C4029D
:105D700089238093C40213C08D3F21F48091BD021A
:105D80008E7F0BC08E3F21F48091BD028D7F05C0B8
:105D90008F3F29F48091BD028B7F8093BD0280915B
:105DA000C502811106C08091C602811102C0109205
:105DB000BE028091C702811106C08091C802811184
:105DC00002C01092BC0208958091BD0280FF08C0FD
:105DD00060910D0170E0759567957595679521C087
:105DE00081FF06C060910D0170E07595679519C03F
:105DF00082FF04C060910D0170E010C09091BC0260
:105E0000992399F060910C019617A0F780910D01EC
:105E1000899FC001112470E00E947A3260387105B8
:105E200040F46115710519F406C061E070E0862F39
:105E300008958FE7089581E008958091BD0280FF65
:105E400006C060910F0170E0660F771F26C081FFCA
:105E500004C060910F0184E005C082FF07C060911B
:105E60000F0188E0689FB001112417C09091BE0215
:105E70009923D1F060910E01961788F720910F01B8
:105E800088E0289F90011124929FA001939F500DBC
:105E9000112470E0CA010E947A326038710540F422
:105EA0006115710519F406C068E070E0862F089549
:105EB0008FE7089581E008958D3E21F40E941D2F03
:105EC000819504C08E3E29F40E941D2F8093C60246
:105ED00008958F3E21F40E941D2F819504C0803FBC
:105EE00029F40E941D2F8093C5020895893F19F45B
:105EF0000E94E42E05C08A3F31F40E94E42E819571
:105F00008093C70208958B3F21F40E94E42E81956F
:105F100004C08C3F29F40E94E42E8093C8020895A7
:105F20009FE0980F983078F421E030E0A90102C09A
:105F3000440F551F9A95E2F7CA019091C402892B2C
:105F40008093C40208958D3F21F48091BD02816049
:105F50000BC08E3F21F48091BD02826005C08F3F4F
:105F600029F48091BD0284608093BD02089580E091
:105F700090E00E94491F80E090E00E94331F109241
:105F800038020E94AE14E3ECF2E086E0DF011D92DD
:105F90008A95E9F71092BE021092BC021092BD02DF
:105FA0000C94C12D8F929F92AF92BF92DF92EF928D
:105FB000FF920F931F93CF93DF93809047029090AF
:105FC0004802A0904902B0904A0240913B02509191
:105FD0003C0260913D0270913E02842A952AA62AD5
:105FE000B72ACFE1D0E025E0D22EE92EF12C082F00
:105FF00010E0D501C4010C2E04C0B695A795979565
:1060000087950A94D2F780FD04C0219790F780E02D
:1060100018C0DC9EF001DD9EF00D1124EE0DFF1D79
:10602000EE0FFF1FEE0FFF1FE00FF11FEE0FFF1F20
:10603000E05EFD4F859194910E948B12019729F3A8
:106040008C2FDF91CF911F910F91FF90EF90DF90F8
:10605000BF90AF909F908F900895990F990F890FDF
:10606000682F669566956695982F977085E0689F6E
:10607000B001112440E050E080E0FB01E40FF51F87
:10608000E753FD4F208130E0092E02C03695279559
:106090000A94E2F721703327042E01C0220F0A94DC
:1060A000EAF7822B4F5F5F4F4530510531F7089576
:1060B000990F990F890FE82FE695E695E695877079
:1060C00051E001C0550F8A95EAF785E0E89FF0019D
:1060D0001124E753FD4F20E030E070E04081CB0118
:1060E000022E02C0969587950A94E2F781708195F9
:1060F00084278523842781932F5F3F4F25303105E7
:1061000069F70895609347027093480280934902AB
:1061100090934A020C94B72F0F931F9341E050E0E5
:1061200060E070E004C0440F551F661F771F8A951A
:10613000D2F7409550956095709580914702909167
:106140004802A0914902B0914A028A019B010823AA
:1061500019232A233B23C901B8011F910F910C94E5
:1061600082300F931F9341E050E060E070E004C084
:10617000440F551F661F771F8A95D2F780914702FB
:1061800090914802A0914902B0914A028A019B0174
:10619000082B192B2A2B3B2BC901B8011F910F91FA
:1061A0000C94823060933B0270933C0280933D02DA
:1061B00090933E020C94B72FFC01808191810E9444
:1061C000EA1592959F70963079F010F4925001C0C4
:1061D0009A50923068F4803F69F018F4883E40F499
:1061E00009C0843F29F406C0883E20F0813F11F0A9
:1061F00080E0089581E008951092390286E0E1EF91
:10620000F1E0DF011D928A95E9F70C94B72F8823FE
:1062100021F00E94A7140C94AE140895882339F03D
:1062200090913902892B809339020C94AE14089511
:106230008823A9F19CEF980F913A60F4EFEEF1E01A
:106240009281891301C01282319691E0E53FF907EE
:10625000B9F70DC090E2980F983058F4877091E02C
:1062600001C0990F8A95EAF7892F0E94A7140C9410
:10627000AE149BE5980F933020F480E090E00C94EE
:10628000491F98E5980F973120F480E090E00C9436
:10629000331F8D3E20F00E946D2E0C94C12D089569
:1062A000CF93882309F49EC0C82F8CEF8C0F813ABE
:1062B00008F043C080915B02813081F030F0823081
:1062C000A1F58C2FCF910C94F61F80913902823268
:1062D00009F06AC08C2F0E9413212CC080913902D2
:1062E0008232C1F3C431C9F058F4CB3069F0C03107
:1062F000B9F482E080935B0288E30E94F61F52C0EB
:10630000C93259F0C83361F48AEA97E00E9447081D
:106310008DEF9FE00E94470845C010925B0208C0C5
:106320008BEF9FE00E94470803C010925B023CC0C5
:1063300080E08170811156C037C080E28C0F8830B8
:1063400078F4C77081E090E001C0880FCA95EAF741
:1063500090913902892B80933902CF910C94AE141D
:10636000EBE5EC0FE33040F4F0E0EF5DFE4F8081B1
:1063700090E0CF910C94491FE8E5EC0FE73150F421
:10638000F0E0EE0FFF1FEC5DFE4F80819181CF9119
:106390000C94331FCD3E30F18C2F0E945C2FCF9197
:1063A0000C94C12D81E0C5CFE1EFF1E087EF91E0E2
:1063B0002191C21721F08E179F07D1F70DC0EFEE84
:1063C000F1E08281C81301C01282319681E0E53F7D
:1063D000F807B9F70E94AE146C2F8FEE91E00E947F
:1063E000191FBBCFCF910895F999FECF92BD81BD02
:1063F000F89A992780B50895A6E1B0E044E050E00E
:106400000C942E32A8E1B0E042E050E00C942E3221
:10641000262FF999FECF92BD81BDF89A019700B45D
:10642000021639F01FBA20BD0FB6F894FA9AF99AFD
:106430000FBE08950396272F0E9409320E9408324A
:10644000252F0E940932242F0C9409320196272F00
:106450000E9409320C940832DC01CB01FC01F9994D
:10646000FECF06C0F2BDE1BDF89A319600B40D92A0
:1064700041505040B8F70895DB018F939F930E94DD
:10648000D432BF91AF91A29F800D911DA39F900D1B
:10649000B29F900D11240895991B79E004C0991FB3
:1064A000961708F0961B881F7A95C9F7809508956E
:1064B00087FB082E062687FD819567FD61950E9462
:1064C0004C320EF4919507FC81950895AA1BBB1BD5
:1064D00051E107C0AA1FBB1FA617B70710F0A61BE4
:1064E000B70B881F991F5A95A9F780959095BC0105
:1064F000CD01089597FB072E16F4009407D077FD81
:1065000009D00E94663207FC05D03EF49095819533
:106510009F4F0895709561957F4F0895A1E21A2EBF
:10652000AA1BBB1BFD010DC0AA1FBB1FEE1FFF1F37
:10653000A217B307E407F50720F0A21BB30BE40B87
:10654000F50B661F771F881F991F1A9469F76095CE
:106550007095809590959B01AC01BD01CF01089588
:10656000EE0FFF1F0590F491E02D09940E94BE32BA
:10657000332312F48A1B9B0B0C94CF32A29FB001E1
:10658000B39FC001A39F700D811D1124911DB29F67
:10659000700D811D1124911D08950E94BE32B7FF18
:1065A0000895821B930B08950E94BE32A59F900D03
:1065B000B49F900DA49F800D911D11240895B7FFE5
:1065C0000C94D4320E94D432821B930B0895FC01A8
:1065D0004150504030F001900616D1F73197CF016D
:1065E0000895882799270895FB01DC0104C08D9147
:1065F0000190801921F441505040C8F7881B990B35
:066600000895F894FFCF9D
:106606007B1C331D141D101D0C1D7A1C28081E0A28
:1066160014010101191A1B1C1D1E1F202122010233
:1066260001818283E200E900EA00B500B600B70006
:10663600CD008301CC008A0192019401210223023C
:1066460024022502260227022A02B300B4006F00A4
:1066560070009196973435679492903F3F3F006D56
:106666006B5F64656C6179006D6B5F696E746572F2
:1066760076616C006D6B5F6D61785F7370656564E4
:10668600006D6B5F74696D655F746F5F6D61780037
:106696006D6B5F776865656C5F6D61785F7370655C
:1066A6006564006D6B5F776865656C5F74696D65C1
:1066B6005F746F5F6D617800407B22D60B5B0B3990
:1066C6000B3C0C550C6E0C0001020202020606067B
:1066D6000909090909090F0F0F0F0F0F15151518CD
:0C66E60019191919191919191919232467
:00000001FF
